:020000040000FA
:06000000EFEF0EF012000C
:06080000EFEF0EF0120004
:06082A000100121E000097
:0808300000010000ED000000D2
:08083800D9CFE6FFE1CFD9FFA3
:10084000040EE126DE6ADE6ADE6ADD6ADD52DD5212
:10085000FD0EDBCF00F0FE0EDBCF01F0026A036A73
:1008600001AE02D002680368D9CFE9FFDACFEAFF10
:10087000030EEB500318E8AE02D0033408D000504A
:10088000EE5C0150EE580250EE580350EE580FE265
:100890000C0EE66ECFEC0EF0E552D9CFE9FFDACFC1
:1008A000EAFFEE2A000EEE22EE22EE22D1D7040E4F
:1008B000E15C02E2E16AE552E16EE552E7CFD9FF81
:1008C00012000F0EC16E070EB46E936A816A300E6D
:1008D000926E80900F0E946EF19E1200D9CFE6FFBB
:1008E000E1CFD9FF020EE1268250020B01E0010E9A
:1008F000080DF3CF02F08250010B040DF3CF01F08D
:100900008050200B01E0010EE824006E8050100B97
:1009100001E0010E002401240224DE6EDD6ADECF38
:1009200000F0DDCF01F000C0F3FF01C0F4FF020EC4
:10093000E15C03E200D0E16AE552E16EE552E7CF07
:10094000D9FF12008092320EE66EFDEC0EF0E552F9
:100950008084320EE66EFDEC0EF0E5528094320E8D
:10096000E66EFDEC0EF0E55212008082010EE66E9E
:10097000E66A62DFE552E5528084010EE66EE66AC1
:100980005BDFE552E5528094010EE66EE66A54DFC5
:10099000E552E5521200380E816ED4DF320EE66E5B
:1009A000E66A4ADFE552E552010E816ECBDF320E78
:1009B000E66EE66A41DFE552E5520D0E816EC2DF5A
:1009C000320EE66EE66A38DFE552E552060E816EBB
:1009D000B9DF320EE66EE66A2FDFE552E55212000D
:1009E000010E816EAFDF0A0EE66EE66A25DFE55284
:1009F000E5521200D9CFE6FFE1CFD9FF020E816E9A
:100A0000A1DF0A0EE66EE66A17DFE552E552FD0E3B
:100A1000DBCFE6FFFE0EDB50280DF350E552E72456
:100A2000E76EFE0EE7CFDBFFFD0EDB6AFE0EDB504E
:100A3000F36EFD0EDBCFF4FFF350F45C0BE2140E0B
:100A4000816E80DF320EE66EFDEC0EF0E552FD0E9B
:100A5000DB2AECD7E552E7CFD9FF1200D9CFE6FF6A
:100A6000E1CFD9FFFE0EDB50816E7FDF010EE66E17
:100A7000E66AE2DEE552E552E552E7CFD9FF120021
:100A8000D9CFE6FFE1CFD9FFFD0EDBCFE9FFFE0EA8
:100A9000DBCFEAFFEF500EE0FD0EDBCFE9FFDB2AF4
:100AA000FE0EDBCFEAFF01E3DB2AEF50E66ED6DF76
:100AB000E552EAD7E552E7CFD9FF12000201046BF5
:100AC000300E926EF00E936EEF0E006F00C281FF3B
:100AD000040E016F0151000821E20051FE0BE842B3
:100AE000006F00C281FF050EE66EE66AA5DEE552E4
:100AF000E5528150100B09E08150200B06E0815037
:100B0000400B03E08150800B01E10AD8020104058B
:100B100002E1055104D00105016FDCD7CFD71200E7
:100B2000F00E936E81CF03F202010315026F0F0ED8
:100B30000015006F00510211006F81CF03F2F00E1B
:100B40000315026FF00E025D01E0F7D7936A06D835
:100B500006C205F20201010E046F12000201076BCA
:100B6000100E075D14E20751EA6A000FE96E010EEC
:100B7000EA22EF50005D08E10751EA6A100FE96EC2
:100B8000010EEA22EFCF06F20729076FE9D706C266
:100B900081FF640EE66EE66A4FDEE552E552120012
:100BA0000201086B070E085D1DE288DF0201096F74
:100BB0000851EA6A0A0FE96E020EEA2209C2EFFF43
:100BC0000851EA6A0A0FE96E020EEA22EF5046085F
:100BD00002E108D004D009C2E6FF40DFE55202017D
:100BE000082BE0D70851EA6A0A0FE96E020EEA22E2
:100BF000EF6A12000201086B070E085D16E2085149
:100C0000EA6A0A0FE96E020EEA22EF50E66E26DF6C
:100C1000E55202010829EA6A0A0FE96E020EEA2289
:100C2000EF5001E102D0082BE7D71200D9CFE6FF41
:100C3000E1CFD9FFE652F250800B01E0010EDF6EEA
:100C4000F29EA69EA69CA684FE0EDB50A96EFD0E0B
:100C5000DB50A86E550EA76EAA0EA76EA682A6B28E
:100C6000FED7A694DF50E8B0F28EE8A0F29EE552DF
:100C7000E552E7CFD9FF1200D9CFE6FFE1CFD9FF88
:100C8000A69CA69EFE0EDB50A96EA680A85000D0A2
:100C9000E552E7CFD9FF1200D9CFE6FFE1CFD9FF68
:100CA000020EE126DE6ADD6ADECF00F0DDCF01F064
:100CB000D890015004E6050E005C000E015824E2B5
:100CC000FD0EDBCF00F0FE0EDBCF01F0DE50002486
:100CD000E96EDD500120EA6EEF50E66EDE50010154
:100CE00020250F01E96EDD50010121210F01EA6E7F
:100CF000170EE926020EEA22E552E750EF6EDF2AD0
:100D0000010E01E3DB2AD0D7050E01012025206F5B
:100D1000000E2121216F020EE15C02E2E16AE55240
:100D2000E16EE552E7CFD9FF1200D9CFE6FFE1CF60
:100D3000D9FF070EE126FE0EDB50280A02E1EAEF9A
:100D40000DF0070A02E1BEEF0DF0090A02E192EF91
:100D50000DF0030A02E166EF0DF01C0A02E13AEF22
:100D60000DF0010A02E10EEF0DF00F0A02E1E2EFD1
:100D70000CF0010A02E1B6EF0CF0030A02E18AEF7F
:100D80000CF0010A02E15EEF0CF0070A02E132EF1B
:100D90000CF0010A02E106EF0CF0030A02E1DAEFBF
:100DA0000BF0010A02E1AEEF0BF06A0A02E182EFFA
:100DB0000BF0030A02E156EF0BF0010A02E12AEF01
:100DC0000BF00F0A02E1FEEF0AF0010A01E1EAD39B
:100DD000030A01E1BBD3010A01E18CD3070A01E157
:100DE0005DD3010A01E12ED3030A01E1FFD2010A1A
:100DF00001E1CFD21F0A01E19FD2010A01E16FD2C6
:100E0000030A01E13FD2010A01E10FD2070A01E121
:100E1000DFD1010A01E1AFD1030A01E17FD1010A6B
:100E200001E14FD10F0A01E11FD1010A01E1EFD029
:100E3000030A01E1BFD0010A01E18FD0070A60E097
:100E4000010A31E0030A02E016EF0EF0DE6ADD6A05
:100E5000DECF00F0DDCF01F0D890015004E6050EA2
:100E6000005C000E01581DE2DECFE9FFDDCFEAFF96
:100E7000250EE926010EEA22EF50E66ED950020F48
:100E8000006EDACF01F0DE500024E96EDD50012063
:100E9000EA6EE552E750EF6EDF2A010E01E3DB2A2E
:100EA000D7D716EF0EF0DE6ADD6ADECF00F0DDCFB9
:100EB00001F0D890015004E6050E005C000E0158C8
:100EC0001DE2DECFE9FFDDCFEAFF2A0EE926010EA3
:100ED000EA22EF50E66ED950020F006EDACF01F031
:100EE000DE500024E96EDD500120EA6EE552E75045
:100EF000EF6EDF2A010E01E3DB2AD7D716EF0EF0E3
:100F0000DE6ADD6ADECF00F0DDCF01F0D89001505F
:100F100004E6050E005C000E01581DE2DECFE9FF7D
:100F2000DDCFEAFF2F0EE926010EEA22EF50E66E32
:100F3000D950020F006EDACF01F0DE500024E96EC6
:100F4000DD500120EA6EE552E750EF6EDF2A010E18
:100F500001E3DB2AD7D716EF0EF0DE6ADD6ADECFBB
:100F600000F0DDCF01F0D890015004E6050E005CE2
:100F7000000E01581DE2DECFE9FFDDCFEAFF340E9F
:100F8000E926010EEA22EF50E66ED950020F006EFC
:100F9000DACF01F0DE500024E96EDD500120EA6E68
:100FA000E552E750EF6EDF2A010E01E3DB2AD7D7C7
:100FB00016EF0EF0DE6ADD6ADECF00F0DDCF01F065
:100FC000D890015004E6050E005C000E01581DE2A9
:100FD000DECFE9FFDDCFEAFF390EE926010EEA2276
:100FE000EF50E66ED950020F006EDACF01F0DE50FE
:100FF0000024E96EDD500120EA6EE552E750EF6E05
:10100000DF2A010E01E3DB2AD7D716EF0EF0DE6AE6
:10101000DD6ADECF00F0DDCF01F0D890015004E6AC
:10102000050E005C000E01581DE2DECFE9FFDDCFAA
:10103000EAFF3E0EE926010EEA22EF50E66ED95095
:10104000020F006EDACF01F0DE500024E96EDD50B1
:101050000120EA6EE552E750EF6EDF2A010E01E350
:10106000DB2AD7D716EF0EF0DE6ADD6ADECF00F09E
:10107000DDCF01F0D890015004E6050E005C000EB3
:1010800001581DE2DECFE9FFDDCFEAFF430EE9267E
:10109000010EEA22EF50E66ED950020F006EDACF51
:1010A00001F0DE500024E96EDD500120EA6EE552C9
:1010B000E750EF6EDF2A010E01E3DB2AD7D716EFE8
:1010C0000EF0DE6ADD6ADECF00F0DDCF01F0D890F1
:1010D000015004E6050E005C000E01581DE2DECF53
:1010E000E9FFDDCFEAFF480EE926010EEA22EF50C4
:1010F000E66ED950020F006EDACF01F0DE50002408
:10110000E96EDD500120EA6EE552E750EF6EDF2A0E
:10111000010E01E3DB2AD7D716EF0EF0DE6ADD6A97
:10112000DECF00F0DDCF01F0D890015004E6050ECF
:10113000005C000E01581DE2DECFE9FFDDCFEAFFC3
:101140004D0EE926010EEA22EF50E66ED950020F4D
:10115000006EDACF01F0DE500024E96EDD50012090
:10116000EA6EE552E750EF6EDF2A010E01E3DB2A5B
:10117000D7D716EF0EF0DE6ADD6ADECF00F0DDCFE6
:1011800001F0D890015004E6050E005C000E0158F5
:101190001DE2DECFE9FFDDCFEAFF520EE926010EA8
:1011A000EA22EF50E66ED950020F006EDACF01F05E
:1011B000DE500024E96EDD500120EA6EE552E75072
:1011C000EF6EDF2A010E01E3DB2AD7D716EF0EF010
:1011D000DE6ADD6ADECF00F0DDCF01F0D89001508D
:1011E00004E6050E005C000E01581DE2DECFE9FFAB
:1011F000DDCFEAFF570EE926010EEA22EF50E66E38
:10120000D950020F006EDACF01F0DE500024E96EF3
:10121000DD500120EA6EE552E750EF6EDF2A010E45
:1012200001E3DB2AD7D716EF0EF0DE6ADD6ADECFE8
:1012300000F0DDCF01F0D890015004E6050E005C0F
:10124000000E01581DE2DECFE9FFDDCFEAFF5C0EA4
:10125000E926010EEA22EF50E66ED950020F006E29
:10126000DACF01F0DE500024E96EDD500120EA6E95
:10127000E552E750EF6EDF2A010E01E3DB2AD7D7F4
:1012800016EF0EF0DE6ADD6ADECF00F0DDCF01F092
:10129000D890015004E6050E005C000E01581DE2D6
:1012A000DECFE9FFDDCFEAFF610EE926010EEA227B
:1012B000EF50E66ED950020F006EDACF01F0DE502B
:1012C0000024E96EDD500120EA6EE552E750EF6E32
:1012D000DF2A010E01E3DB2AD7D716EF0EF0DE6A14
:1012E000DD6ADECF00F0DDCF01F0D890015004E6DA
:1012F000050E005C000E01581DE2DECFE9FFDDCFD8
:10130000EAFF660EE926010EEA22EF50E66ED9509A
:10131000020F006EDACF01F0DE500024E96EDD50DE
:101320000120EA6EE552E750EF6EDF2A010E01E37D
:10133000DB2AD7D716EF0EF0DE6ADD6ADECF00F0CB
:10134000DDCF01F0D890015004E6050E005C000EE0
:1013500001581DE2DECFE9FFDDCFEAFF6B0EE92683
:10136000010EEA22EF50E66ED950020F006EDACF7E
:1013700001F0DE500024E96EDD500120EA6EE552F6
:10138000E750EF6EDF2A010E01E3DB2AD7D716EF15
:101390000EF0DE6ADD6ADECF00F0DDCF01F0D8901E
:1013A000015004E6050E005C000E01581DE2DECF80
:1013B000E9FFDDCFEAFF700EE926010EEA22EF50C9
:1013C000E66ED950020F006EDACF01F0DE50002435
:1013D000E96EDD500120EA6EE552E750EF6EDF2A3C
:1013E000010E01E3DB2AD7D716EF0EF0DE6ADD6AC5
:1013F000DECF00F0DDCF01F0D890015004E6050EFD
:10140000005C000E01581DE2DECFE9FFDDCFEAFFF0
:10141000750EE926010EEA22EF50E66ED950020F52
:10142000006EDACF01F0DE500024E96EDD500120BD
:10143000EA6EE552E750EF6EDF2A010E01E3DB2A88
:10144000D7D7F4D3DE6ADD6ADECF00F0DDCF01F05E
:10145000D890015004E6050E005C000E01581DE214
:10146000DECFE9FFDDCFEAFF7A0EE926010EEA22A0
:10147000EF50E66ED950020F006EDACF01F0DE5069
:101480000024E96EDD500120EA6EE552E750EF6E70
:10149000DF2A010E01E3DB2AD7D7C8D3DE6ADD6A73
:1014A000DECF00F0DDCF01F0D890015004E6050E4C
:1014B000005C000E01581DE2DECFE9FFDDCFEAFF40
:1014C0007F0EE926010EEA22EF50E66ED950020F98
:1014D000006EDACF01F0DE500024E96EDD5001200D
:1014E000EA6EE552E750EF6EDF2A010E01E3DB2AD8
:1014F000D7D79CD3DE6ADD6ADECF00F0DDCF01F006
:10150000D890015004E6050E005C000E01581DE263
:10151000DECFE9FFDDCFEAFF840EE926010EEA22E5
:10152000EF50E66ED950020F006EDACF01F0DE50B8
:101530000024E96EDD500120EA6EE552E750EF6EBF
:10154000DF2A010E01E3DB2AD7D770D3DE6ADD6A1A
:10155000DECF00F0DDCF01F0D890015004E6050E9B
:10156000005C000E01581DE2DECFE9FFDDCFEAFF8F
:10157000890EE926010EEA22EF50E66ED950020FDD
:10158000006EDACF01F0DE500024E96EDD5001205C
:10159000EA6EE552E750EF6EDF2A010E01E3DB2A27
:1015A000D7D744D3DE6ADD6ADECF00F0DDCF01F0AD
:1015B000D890015004E6050E005C000E01581DE2B3
:1015C000DECFE9FFDDCFEAFF8E0EE926010EEA222B
:1015D000EF50E66ED950020F006EDACF01F0DE5008
:1015E0000024E96EDD500120EA6EE552E750EF6E0F
:1015F000DF2A010E01E3DB2AD7D718D3DE6ADD6AC2
:10160000DECF00F0DDCF01F0D890015004E6050EEA
:10161000005C000E01581DE2DECFE9FFDDCFEAFFDE
:10162000930EE926010EEA22EF50E66ED950020F22
:10163000006EDACF01F0DE500024E96EDD500120AB
:10164000EA6EE552E750EF6EDF2A010E01E3DB2A76
:10165000D7D7ECD2DE6ADD6ADECF00F0DDCF01F055
:10166000D890015004E6050E005C000E01581DE202
:10167000DECFE9FFDDCFEAFF980EE926010EEA2270
:10168000EF50E66ED950020F006EDACF01F0DE5057
:101690000024E96EDD500120EA6EE552E750EF6E5E
:1016A000DF2A010E01E3DB2AD7D7C0D2DE6ADD6A6A
:1016B000DECF00F0DDCF01F0D890015004E6050E3A
:1016C000005C000E01581DE2DECFE9FFDDCFEAFF2E
:1016D0009D0EE926010EEA22EF50E66ED950020F68
:1016E000006EDACF01F0DE500024E96EDD500120FB
:1016F000EA6EE552E750EF6EDF2A010E01E3DB2AC6
:10170000D7D794D2DE6ADD6ADECF00F0DDCF01F0FC
:10171000D890015004E6050E005C000E01581DE251
:10172000DECFE9FFDDCFEAFFA20EE926010EEA22B5
:10173000EF50E66ED950020F006EDACF01F0DE50A6
:101740000024E96EDD500120EA6EE552E750EF6EAD
:10175000DF2A010E01E3DB2AD7D768D2DE6ADD6A11
:10176000DECF00F0DDCF01F0D890015004E6050E89
:10177000005C000E01581DE2DECFE9FFDDCFEAFF7D
:10178000A70EE926010EEA22EF50E66ED950020FAD
:10179000006EDACF01F0DE500024E96EDD5001204A
:1017A000EA6EE552E750EF6EDF2A010E01E3DB2A15
:1017B000D7D73CD2DE6ADD6ADECF00F0DDCF01F0A4
:1017C000D890015004E6050E005C000E01581DE2A1
:1017D000DECFE9FFDDCFEAFFAC0EE926010EEA22FB
:1017E000EF50E66ED950020F006EDACF01F0DE50F6
:1017F0000024E96EDD500120EA6EE552E750EF6EFD
:10180000DF2A010E01E3DB2AD7D710D2DE6ADD6AB8
:10181000DECF00F0DDCF01F0D890015004E6050ED8
:10182000005C000E01581DE2DECFE9FFDDCFEAFFCC
:10183000B10EE926010EEA22EF50E66ED950020FF2
:10184000006EDACF01F0DE500024E96EDD50012099
:10185000EA6EE552E750EF6EDF2A010E01E3DB2A64
:10186000D7D7E4D1DE6ADD6ADECF00F0DDCF01F04C
:10187000D890015004E6050E005C000E01581DE2F0
:10188000DECFE9FFDDCFEAFFB60EE926010EEA2240
:10189000EF50E66ED950020F006EDACF01F0DE5045
:1018A0000024E96EDD500120EA6EE552E750EF6E4C
:1018B000DF2A010E01E3DB2AD7D7B8D1DE6ADD6A61
:1018C000DECF00F0DDCF01F0D890015004E6050E28
:1018D000005C000E01581DE2DECFE9FFDDCFEAFF1C
:1018E000BB0EE926010EEA22EF50E66ED950020F38
:1018F000006EDACF01F0DE500024E96EDD500120E9
:10190000EA6EE552E750EF6EDF2A010E01E3DB2AB3
:10191000D7D78CD1DE6ADD6ADECF00F0DDCF01F0F3
:10192000D890015004E6050E005C000E01581DE23F
:10193000DECFE9FFDDCFEAFFC00EE926010EEA2285
:10194000EF50E66ED950020F006EDACF01F0DE5094
:101950000024E96EDD500120EA6EE552E750EF6E9B
:10196000DF2A010E01E3DB2AD7D760D1DE6ADD6A08
:10197000DECF00F0DDCF01F0D890015004E6050E77
:10198000005C000E01581DE2DECFE9FFDDCFEAFF6B
:10199000C50EE926010EEA22EF50E66ED950020F7D
:1019A000006EDACF01F0DE500024E96EDD50012038
:1019B000EA6EE552E750EF6EDF2A010E01E3DB2A03
:1019C000D7D734D1DE6ADD6ADECF00F0DDCF01F09B
:1019D000D890015004E6050E005C000E01581DE28F
:1019E000DECFE9FFDDCFEAFFCA0EE926010EEA22CB
:1019F000EF50E66ED950020F006EDACF01F0DE50E4
:101A00000024E96EDD500120EA6EE552E750EF6EEA
:101A1000DF2A010E01E3DB2AD7D708D1DE6ADD6AAF
:101A2000DECF00F0DDCF01F0D890015004E6050EC6
:101A3000005C000E01581DE2DECFE9FFDDCFEAFFBA
:101A4000CF0EE926010EEA22EF50E66ED950020FC2
:101A5000006EDACF01F0DE500024E96EDD50012087
:101A6000EA6EE552E750EF6EDF2A010E01E3DB2A52
:101A7000D7D7DCD0DE6ADD6ADECF00F0DDCF01F043
:101A8000D890015004E6050E005C000E01581DE2DE
:101A9000DECFE9FFDDCFEAFFD40EE926010EEA2210
:101AA000EF50E66ED950020F006EDACF01F0DE5033
:101AB0000024E96EDD500120EA6EE552E750EF6E3A
:101AC000DF2A010E01E3DB2AD7D7B0D0DE6ADD6A58
:101AD000DECF00F0DDCF01F0D890015004E6050E16
:101AE000005C000E01581DE2DECFE9FFDDCFEAFF0A
:101AF000D90EE926010EEA22EF50E66ED950020F08
:101B0000006EDACF01F0DE500024E96EDD500120D6
:101B1000EA6EE552E750EF6EDF2A010E01E3DB2AA1
:101B2000D7D784D0DE6ADD6ADECF00F0DDCF01F0EA
:101B3000D890015004E6050E005C000E01581DE22D
:101B4000DECFE9FFDDCFEAFFDE0EE926010EEA2255
:101B5000EF50E66ED950020F006EDACF01F0DE5082
:101B60000024E96EDD500120EA6EE552E750EF6E89
:101B7000DF2A010E01E3DB2AD7D758D0DE6ADD6AFF
:101B8000DECF00F0DDCF01F0D890015004E6050E65
:101B9000005C000E01581DE2DECFE9FFDDCFEAFF59
:101BA000E30EE926010EEA22EF50E66ED950020F4D
:101BB000006EDACF01F0DE500024E96EDD50012026
:101BC000EA6EE552E750EF6EDF2A010E01E3DB2AF1
:101BD000D7D72CD0DE6ADD6ADECF00F0DDCF01F092
:101BE000D890015004E6050E005C000E01581DE27D
:101BF000DECFE9FFDDCFEAFFE80EE926010EEA229B
:101C0000EF50E66ED950020F006EDACF01F0DE50D1
:101C10000024E96EDD500120EA6EE552E750EF6ED8
:101C2000DF2A010E01E3DB2AD7D700D0D950020FFB
:101C3000E66E000EDA20E66E4CEC06F0E552E55258
:101C4000070EE15C02E2E16AE552E16EE552E7CFA0
:101C5000D9FF120061EC04F00201156B166B020E45
:101C600016AF02D0D89003D0155D000E165910E2C1
:101C7000220E1525E96E010E1621EA6EEF50E66E72
:101C800095EC06F0E5520201152B000E1623E7D75E
:101C9000136B146B806A80820A0EE66EFDEC0EF008
:101CA000E55280920201136B146B0A0E14AF02D03E
:101CB000D89003D0135D000E145920E2170E13259F
:101CC000E96E020E1421EA6EEF50816E020EE66E8E
:101CD000E66A1CEC04F0E552E55280840A0EE66EDA
:101CE000FDEC0EF0E55280940A0EE66EFDEC0EF06F
:101CF000E5520201132B000E1423D7D7C9D71200C7
:101D00002A0EF66E080EF76E000EF86E010109003D
:101D1000F550F26F0900F550F36F03E1F26701D05F
:101D20003DD00900F550ED6F0900F550EE6F090048
:101D3000F550EF6F09000900F550E96E0900F55004
:101D4000EA6E090009000900F550F06F0900F5502E
:101D5000F16F09000900F6CFF4F1F7CFF5F1F8CFF4
:101D6000F6F1EDC1F6FFEEC1F7FFEFC1F8FF01019B
:101D7000F05302E1F15307E00900F550EE6EF00771
:101D8000F8E2F107F9D7F4C1F6FFF5C1F7FFF6C1A4
:0E1D9000F8FF0101F207000EF35BBFD712004F
:021D9E00FF0E36
:101DA000E350066E480E01D04C0EE76EE72EFED7CC
:0E1DB000E76AE72EFED7062EF7D700001200D6
:021DBE00000E15
:101DC000F36E00EE00F0080E01D81200EA6002D0B7
:0E1DD000EE6AFCD7F350E9601200EE6AFCD711
:021DDE0012EE03
:101DE00040F022EE40F0F86A059C80EC0EF008EC22
:0A1DF0000FF02AEC0EF0FBD71200F2
:061DFA00FF0EE350E84E6D
:101E00001200000000D000D000D0E82EFAD7120057
:021E10001200BE
:0E1E1200EEEDEBE7DEDDDBD7BEBDBBB77E7DC0
:101E20007B773031323334353637383941424344A9
:101E300045460000252600FC121212FCFE929292EA
:101E40006C7C82828244FE8282827CFE92929282AA
:101E5000FE121212027C92929274FE101010FE007A
:101E600082FE8200708080807EFE10284482FE8088
:101E7000808080FE041804FEFE081020FE7C828212
:101E8000827CFE1212120CFC82A242BCFE12325262
:101E90008C4C929292640202FE02027E8080807ECE
:101EA0003E4080403EFE403040FEC6281028C60618
:101EB00008F00806C2A2928A867C8282827C008414
:101EC000FE800084C2A2928C448292926C1E1010FA
:101ED00010FE5E929292627C9292926482422212F0
:101EE0000E6C9292926C4C9292927C000C1E3E7CF4
:0F1EF0003E1E0C000010387CFE38383838383869
:00000001FF
